:10000000012883160430850001308600C03081004D
:1000100006309F00831200309200E1202C211B212A
:10002000B201643044216430442106308A004C28F7
:100030002020D100162108002020D200162108001F
:100040000830AE00C0018515043006210310C00C35
:1000500005160519C017051206300621AE0B262815
:10006000400885110800831307308A005208B03E0B
:1000700003188317031C52088400A0300318203093
:10008000840751087F39E020D11B80005A300721B6
:1000900006308A0016210800EE2033300721162191
:1000A00018201C2033202630A20000005F300521DC
:1000B0001621A20B5528A030A3008313B530A2004F
:1000C000A501A50AAB0157300621043005211621F0
:1000D0000430052125085F3A031D74280000AB0198
:1000E0002030A300831779280000000000000000E2
:1000F0007928230884002B08063C031C8128A120B2
:100100008428000048300521251CAB0A2B080C3A36
:10011000031D8E28AB011430A307912800000000B6
:1001200091280000A50AA20B6528073006211B3084
:10013000A20016215F300721A20B992816210B215E
:100140004C28DD2093000000DD2093000000DD201E
:1001500093000000DD2093000000DD2093000000EC
:10016000DD2093000000DD2093000000DD209300DF
:100170000000DD2093000000DD2093000000DD2062
:1001800093000000DD2093000000DD2093000000BC
:10019000DD2093000000DD2093000000DD209300AF
:1001A0000000DD2093000000DD2093000000DD2032
:1001B00093000000DD20930008000008840A2B074C
:1001C000820083168030940083122030940008004F
:1001D0008316141CE9288312930008000630B5002A
:1001E00016212B300721B50BF0280730B50011215F
:1001F0002B300721B50BF7280630B5001121162149
:100200002B300721B50BFF28080000000000B100CB
:10021000B10B08290800000000005F300F290721FA
:100220000800861504300721861108008611043065
:1002300007218615080007308A0083165630E02013
:10024000A0003130E020A1003230E020A2003230A6
:10025000E020A300831208008313A0308400203024
:100260003821831720308400203038218313080080
:10027000B5005030AE0007308A003508E02080001D
:10028000840AAE0B3D290800A8005321A80B45297C
:1002900008000130542902305429053054290A300D
:1002A0005429323054296430A700000000000000B7
:0E02B0000E30A600A60B5A29A70B55290800F0
:100C0000FC3482348234FC3482348234FC348034C8
:100C1000803480347C348234803480348034823434
:100C20007C348234803480348E3482347C34FE349C
:100C300080348034FE3480348034FE348034803418
:100C40008034803480348034FE34103410341034D6
:100C50001034103410341034383444348234823434
:100C6000FE34823482348234FE34823482348234DC
:100C70008234823482347C34823480347C34023452
:100C800082347C34823402343C3440348034FE3448
:100C90000234043408341034303410341034103436
:100CA000103410347C34823402340C3402348234F4
:100CB0007C34823482347C34823482347E34023414
:100CC00002347C34FC348234823482348234823480
:100CD000FC3482348234FC348234823482342834CA
:100CE000023402347C34823482348234FE3402345E
:100CF000023402340234023482347C347C34823450
:100D00008A349234A23482347C347C34803480340B
:100D1000FC34823482347C34823484348834E03449
:100D20008834843482348234C634AA34923482348F
:100D300082348234823444342834103428344434A5
:100D400082348234C234A23492348A348634823477
:100D5000823482349234AA34C6348234FE34043469
:100D60000834103420344034FE3480348034FC3471
:100D7000023402347C347C348234823482348234CF
:100D800082347C347C348234823482348A348634B3
:100D90007C3482340234043408340034083400349F
:100DA0000034003400340034003400341834183473
:100DB000003418341834003400347C3400347C346B
:100DC0000034003400347C34003400340034023405
:100DD00004340834103420344034003410341034D7
:100DE000FE34103410340034023406340E341E3411
:060DF0000E34063402344B
:100E0000CF34CF34CF34CF34CF34CF34CF34CF34CA
:100E1000CF34CF34CF34CF34CF34CF34CF34CF34BA
:100E2000CF34CF34CF34CF34CF34CF34CF34CF34AA
:100E3000CF34CF34CF34CF34CF34CF34CF34CF349A
:100E4000CF34CF34CF34CF34CF34CF34CF34CF348A
:100E5000CF34CF34CF34ED34CF34E034D134E63432
:100E60007E344C34413452347334B4348534473492
:100E700058345B34D434CF34F434DB34CF34C83416
:100E8000CF342C3400340A34623417341A3410341A
:100E90003134253477348C341E349334A134BB344C
:100EA0000334C23468343B34243435349734A734A3
:100EB0009A346C34AE34CF34CF34CF34CF34CF34D3
:100EC000CF342C3400340A34623417341A341034DA
:100ED0003134253477348C341E349334A134BB340C
:100EE0000334C23468343B34243435349734A73463
:100EF0009A346C34AE34CF34CF34CF34CF34CF3493
:02400E00222F5F
:00000001FF
